:020000020000FC
:1000000066CEC2C10000000020C0000094C0000005
:1000100000009EC000000000000000000203040673
:10002000080C10182030406080000406080C1018DE
:100030002030406080A0C00000070F1F3F000D0D62
:100040000403060D0503030202004FB662FD0EC055
:10005000552009F00994C52DC095089483FDC795D6
:10006000C4BDC093A10064604FBE1895C0916400E8
:10007000089483FDC795C4BDC093A1006B7FC09158
:100080006400CF3F09F420C070FF02C082FD05C0AC
:100090004FBE919890989398189575FD0EC065FD88
:1000A0000CC0C091B300C0FD9498C1FD9798C2FDEB
:1000B0009598CAEFC095CA95F1F791989098939842
:1000C0002092A1004FBE189524BCCC27C064C8BFA5
:1000D0006460F6CFC0CF70FFBECF65FDBCCF919AF4
:1000E000BACF70FFB8CF65FDB6CF909AB4CF70FF8E
:1000F000B2CF65FDB0CF939AAECF949A70FFABCFDD
:1001000065FDA9CFC7E0CA95F1F7919AA4CF979A58
:1001100070FFA1CF65FD9FCFC7E0CA95F1F7909A18
:100120009ACF959A70FF97CF65FD95CFC7E0CA9596
:10013000F1F7939A90CF4FB6C9B7CF7EC9BF6E7F04
:10014000CCB5CE0DDDB5DF1DDBBDCABD4FBE1895EC
:100150003FB68F7EABB7A074A2118061A0E0ABBFA9
:10016000A9B7AE7FA9BF7894A0916800AA2341F0F7
:1001700085FD2AC0A0916800AA95A093680024C0BC
:1001800040E050E085FD14C0A0B396FDA095A2FD0F
:100190004FEFA3E096FDA2E0A5BFAA27A064AABFE7
:1001A0008D7FA0B396FDA095A2FD5FEF451741F7A7
:1001B000A0E461FDA093680085FD03C0A0E4A093C6
:1001C000680040939700816085FD0EC0A091690092
:1001D000AA2331F0A0916900AA95A093690004C0F8
:1001E0008061AA27A064AABF80FF0AC0A0919700DF
:1001F0004A2F61FF8E7F85FD01C000C040936100E2
:100200004091B600443009F004C0A0916100A09371
:100210006300A52DA03408F06860A0916000A3954C
:10022000A093600051F0F894A9B7A160A9BF84FF22
:1002300002C0A0E4ABBF3FBE1895A0917400A39587
:10024000A093740042E050916800552329F085FF87
:1002500003C05A9550936800A0919700A13018F000
:1002600020929A000DC020929B002092A500A091A0
:100270009A00AF5FA0939A0018F0AFEFA0939A0096
:10028000B09061005091B600523049F466FF91F091
:10029000A2E3BA1678F0A0918700A09361005330D2
:1002A00049F466FF39F0A2E3BA1620F0A091C2002B
:1002B000A0936100509162005B1521F010F05A95F7
:1002C00001C05395509362004A95D1F65091A50014
:1002D000539509F45A955093A500A091A600AA95AC
:1002E000A093A60009F046C0A1E0A093A60045E0B7
:1002F000A091A7005A17F0F1A091A8005A1728F46E
:1003000041E0A3E0A093A60007C0A091A9005A175E
:1003100018F441E04093A600D0909D00C090630087
:10032000DC14A8F0A091B600A430D9F066FD0FC08F
:10033000C0929D00539511F0A091A700A093A50035
:10034000A1E0A093A600ACE3A093620013C0A0912B
:100350009D00A40F20F45FEF50939D0002C0A09376
:100360009D00A0919D00AF3F29F4AFEFA0939B00AB
:10037000A093A500F894A9B7A160A9BF84FF02C00B
:10038000A0E4ABBF3FBE18953FB64CB55DB58F7EC0
:10039000ABB7A074A2118061A0E0ABBFA9B7AE7FDC
:1003A000A9BF789481FD23C0A2E096FDA3E0A5BF7C
:1003B0008260A0B396FDA095A2FF05C040936500A2
:1003C000509366001CC1A3E096FDA2E0A5BFAA273A
:1003D000A064AABF8D7F85FF01C004C140E0A0B327
:1003E00096FDA095A2FDFEC040939700EDC0A3E04E
:1003F00096FDA2E0A5BF8D7F61FF71C0A2E096FDD2
:10040000A3E0A5BFAA27A064AABF82604093920080
:1004100050939300A09090004A19B09091005B090E
:10042000BB24A22C4C38520518F42092960049C0E7
:10043000A091D600AA2359F1483C520528F4A0E126
:10044000BA2EAAE0AA2E23C04836A1E05A0728F403
:10045000A8E0BA2EAFE0AA2E1AC0403DA2E05A078B
:1004600028F4A4E0BA2EAEE1AA2E11C0403AA5E0CD
:100470005A0728F4A2E0BA2EACE3AA2E08C04839E5
:10048000A8E05A0720F4A1E0BA2EA8E7AA2EC42EAD
:10049000A0919400CA1AD52EA0919500DA0ADD2009
:1004A0002AF4AFEFC094D094CA1ADA0A20929600C8
:1004B000A8E0A210A0E0CA14DA0618F4A1E0A09304
:1004C0009600409394005093950040919200509173
:1004D0009300409390005093910002E075C0A0916A
:1004E00065004A1BA09166005A0B94FD60C093FD05
:1004F0005EC092FD5AC086FF03C0D52EC42E0CC02C
:100500005695479591FD51C05695479590FD4DC024
:10051000D52EC42ED694C79461FD19C0AC2DAC5114
:10052000AD2DA24008F005C0DD2089F4AC2DA85CFB
:1005300070F4A0916700A395AA2311F0A09367001F
:10054000AA3008F44FC02092970081604BC0A09160
:100550006700AA2319F0AA95A0936700A22C5091D6
:10056000BC0097FD02C0A090CA00AAEFAA0EA22D5F
:10057000A21DCA18DA0A4FB74170442319F040E0AF
:1005800050E015C0AFEFCA16D20418F04FEF50E09C
:100590000EC0A091AE00CA9E412D000C441F50E039
:1005A00008F012C04FEF50E00FC05695479594FFEA
:1005B00007C0552309F04FEFA42FA6954A0F521DEF
:1005C0004F3F520508F04FEF40939700816061FF65
:1005D00009C0AFE1A095A923AB299A2F8F7DBB203D
:1005E00009F48062A0E4A093680085FF03C0AAE03C
:1005F000A093680061FD03C085FD01C08F7E85FD6D
:1006000003C0A0E2A0936900F894A9B7A160A9BFB4
:1006100084FF02C0A0E4ABBF3FBE189511E00AC042
:1006200013E008C01AE006C01EE104C014E602C0D0
:1006300018EC00C005E1BB27BA95F1F70A95D9F788
:100640001A95C1F708952AE338E709C020E33CE88A
:1006500006C02AE234EB03C025E238EC00C012E009
:1006600095FD9F7D95FF9062BB27979ABA95F1F70C
:10067000909ABA95F1F79098BA95F1F79798BA953C
:10068000F1F7919AB091AF00BA95F1F79198B7E868
:10069000BA95F1F71A9521F7022FB22FBA95F1F713
:1006A0000A95D9F73A95D9F6979A0895221B39E019
:1006B000001F3A9509F40895221F211B18F4210FF9
:1006C0008894F6CF0894F4CF622C722CB0E0889412
:1006D000B395221F331FE0F7379527958894912E05
:1006E000802E020B130B10F4192D082D10F4889492
:1006F00001C00894661C771CBA9571F7172D062D5A
:100700000895322D11232AF43A9500951095031B74
:10071000130BF894029F712C002D129F912C802CAA
:100720007894780C172D921C292DB4E06B2E269509
:10073000179507956A94D9F7332321F00095109502
:10074000031B130B08950091B600043009F474C024
:10075000B0919700B95198F0B72FB67081F466FD4B
:100760002BC005E09090C800B92DBA9521F00AE0A1
:10077000BA9509F002E1B0917B00B01BE0F066FF92
:100780000AC0B0919F00B0939D00BFEFB093A50049
:10079000B1E0B093A600B0916100B09363002092E5
:1007A0007F0020928000209281002092820020927F
:1007B00083006F7B41C060649090C800B92DBA95EA
:1007C00079F4B0916200B095BB1FBB1F1B2FB7958A
:1007D0000B2FB12FB170B3951B2FB02FBE7F25C04B
:1007E000B92DBA95BA9581F4B0916200B095BB1F4E
:1007F000BB1FBB1F1B2FB7950B2FB12FB370B3952A
:100800001B2FB02FBC7F14C0B0916200B095BB1FEE
:10081000BB1FBB1FBB1F1B2FB7950B2FB12FB77073
:10082000B395B3951B2FB02FB87FB0540B2F12097F
:1008300000937F0010938000089510917B0016951F
:1008400000917A000795B0917F00B01B0B2FB091FB
:100850008000B10B1B2F28F40038BFEF1B0740F0BE
:1008600009C00F37120508F405C00FE710E002C0F9
:1008700000E81FEF00938400109385000895009115
:100880008400B09181000B0F10918500B09182001F
:100890001B1F20E03091850033230AF42A95B09184
:1008A00083002B1F1AF4203F40F00AC02F3008F4B9
:1008B00007C00FEF1FEF2FE003C000E010E020EFB4
:1008C00030916300B0919C003B1718F4323030F047
:1008D00009C0B0918500BB235AF004C0B0918500D7
:1008E000BB2332F400938100109382002093830095
:1008F00008952091D80000918400000F1091850088
:10090000111FFFDE11232AF40038BFEF1B0740F050
:1009100009C00F37120508F405C00FE710E002C048
:1009200000E81FEF002352F0B0916200B01B0B2FC4
:1009300018F0013008F00AC001E008C000950F5F10
:10094000B09162000B0F08F001C00FEF009386001A
:1009500008952091D9000091820010918300D1DE8A
:1009600011232AF40130BFEF1B0740F009C00F3FED
:10097000120508F405C00FEF10E002C001E01FEF00
:10098000112352F0B0918600B01B0B2F18F00130EC
:1009900008F00AC001E008C000950F5FB091860022
:1009A0000B0F08F001C00FEF0093630008950FEFE5
:1009B000677F71FD29C072FD09C06860B0917B003E
:1009C000BA3020F0B52DB03408F4677FB091D5006F
:1009D000BB23D1F0B0917B00BB23B1F00FEF10919E
:1009E0007B0064DEF894B091730072FDB5E00B9F5C
:1009F000112D002D7894112309F00FEFB0919F0075
:100A00000B1710F400919F0000939E000895009131
:100A10007A0010917B0000541140B0919E0010F4B8
:100A2000BA9501C0B39511F0B0939E000895F4D328
:100A3000B7E073FDB7E0B06CB7B9B6B1B068B064F9
:100A4000B6B9ECDDB7E073FDB7E0B06CB7B9B6B1DD
:100A5000B068B064B6B9B6B1B6FDFDCF04B115B19A
:100A6000B6B1BF77B6B929D42DE62093AA002223C8
:100A700009F441C030E03093AB00732E7694622EBF
:100A80006694620E731E262D372D0217130778F019
:100A90008090AA00BDE6B80DB093AA008090AB008C
:100AA000B0E0B81DB093AB00260D371DEECF80909F
:100AB000AA009090AB001091AB0016950091AA008F
:100AC00007951695079523E0169507952A95E1F762
:100AD0002091B7002A9529F42092AA002092AB0019
:100AE0000AC02A9521F0800E911E2A95E1F7809286
:100AF000AA009092AB0008952091B700B6B1B6FD60
:100B0000FBCF04B115B1B6B1BF77B6B9B091AC00A7
:100B1000B395B093AC00B83060F12092AC00B091C6
:100B2000D400BB2321F1112329F0B091AD00BF3FC8
:100B300061F009C0B091AD000B1739F020F4BB2370
:100B400021F0BA9502C0B395E1F300919C00B093F7
:100B5000AD00B03050F400ECB03038F400E8B03004
:100B600020F400E4B03008F400E000939C00777FAC
:100B700008952130B1F00F3FB3E01B0790F4BDE6BC
:100B8000BB2379F0B091AA000B17B091AB001B0703
:100B900040F4B0919C00BB2359F0BA95B0939C00EF
:100BA00007C0B0919C00BF3F19F0B395B0939C0073
:100BB00000919C00B0916300B01B10F400916300A1
:100BC000B0919D000B1750F000919D00B0919D00D9
:100BD000BF3F21F0B0919D00B0939C00502E009338
:100BE0006400B091AC00B73009F47860089502E376
:100BF000F894B091DA000B9F012D000C001F78943F
:100C0000B0919C000B1710F000919C0000936100C4
:100C100000936300502E0093640000939F0008959A
:100C200020927A00B0EFB0937B000895F8940CB551
:100C30001DB5209174007894309175006090760015
:100C40000093750010937600031B160971FD03C015
:100C500076FD81C02BC07090770020937700270924
:100C6000222311F00FEF1FEF809078009090790011
:100C700030937800609279006918161910937C00FF
:100C800000917500109176000819190920917A00D9
:100C900030917B0036952795020F131F10F40FEF4C
:100CA0001FEF00937A0010937B0029C020917A00F7
:100CB00030917B003901B4E08B2EB2E09B2E3430B2
:100CC00010F08A949A94383010F08A949A9476941A
:100CD00067948A94E1F726193709992021F016952F
:100CE00007959A94E1F7200F311F20937A003093F3
:100CF0007B0028F43FEF30937A0030937B00323052
:100D000008F4706471FF02C0B3E00DC0B091C6007A
:100D100000917100023838F0B395003A08F0B395AD
:100D2000B63008F0B5E09B2EB4E08B2E10917B001E
:100D300000917A0024E0169507952A95E1F70819A5
:100D4000120928F0B02FB250B12FB20910F402E00E
:100D500010E0980126C020917A0030917B00390183
:100D6000769467946694669466942619320906957B
:100D70000695200F321D20937A0030937B0032308D
:100D800008F07F7B04E036952795369527952695C4
:100D90002695201B10F0223008F422E08901909063
:100DA000C60060FDFECFE0908C00F0908D00616089
:100DB000B9B7B061B9BF380176FD44C07694679485
:100DC00000938C0010938D00B92DB330E1F0B0FD8D
:100DD00004C0060D171D930106C0000F111F02501D
:100DE000120922E030E0B92DB33068F020938E0074
:100DF00030938F00009388001093890060928A00DE
:100E000070928B003DC000938E0010938F00209352
:100E100088003093890060928A0070928B0071FF85
:100E200010C0B0916D00B33060F000918F00109150
:100E30007C001595010F28F022F020928E0000937F
:100E40008F001EC0669400938C00B92DB33091F0D2
:100E5000B0FD03C0060D262D03C0000F025022E096
:100E6000B92DB33038F020938E0000938800609243
:100E70008A0006C000938E002093880060928A004A
:100E800000917D0002FD0350013031F495FD0CC04E
:100E9000B2E0B06CB7B90BC0023021F4B3E0B06C73
:100EA000B7B905C095FDF4CFB4E0B06CB7B9009107
:100EB000A400000F10F4BBE60B270093A40060FD14
:100EC000FECFB2E0B0936E006160B9B7B061B9BF58
:100ED000B72FB670A1F020917A0030917B00369543
:100EE0002795F8940CB51DB5020F131F1BBD0ABD45
:100EF0006160B0E1B8BFB9B7B061B9BF7894089587
:100F0000606120927E0020E067FD20E206C0606103
:100F100020927E0020E267FD20E0789401E076FDDB
:100F200011C0B72FB67009F06F7EB0917B00B5503D
:100F300048F002E0B55020F003E0B55008F006E0BC
:100F400071FD0AE060FD12C0B0917E00BB2371F01C
:100F500071FF08C0B0916D00B33020F0B0916E0009
:100F6000BA9519F4789470615CC0AEDF7894000093
:100F70000000F89476FD16C010917B00173008F041
:100F800017E0B5E01B0F72FD10E183FF110F62FF48
:100F9000110F71FD12E8B4B56090A100B61990F27E
:100FA000B10B80F2B0B7B77FB0BFB8B1B0B7B8601F
:100FB000B0BFB0917E00B395B0937E00B8B176FD1E
:100FC00006C0B1E071FDB2E0BA95F1F7B8B1B07208
:100FD000B21709F01BC071FF05C003950A3008F075
:100FE0000395B0CF64FF99CF6F7E3CB56DB4709020
:100FF0007A0080907B00370D681C6BBC3ABD616045
:10100000B0E1B8BFB9B7B061B9BF87CFB0916D00DB
:10101000B23008F482CF64FD80CF0A9509F092CFF8
:101020007F7E20918E0030918F00F894B0E1B8BFA0
:101030000CB51DB5020F131F1BBD0ABDE090880043
:10104000F09089006160B9B7B061B9BF7894B72FEB
:10105000B67039F0B0916D0072FFB395B0936D002A
:1010600009C074FF07C067FD05C064FD03C0BF91E0
:10107000BF91DCC4089500E063FF03C064FF01C0BA
:1010800001E0F89410917100B7E01B9F212D102D05
:101090007894200F269517952695179526951795E0
:1010A00010937100183718F4B8E7B09371000091ED
:1010B0007100B09172000B1720F0606291989098C7
:1010C000939860FDFECFE0908A00F0908B00616005
:1010D000B9B7B061B9BF0895B2E095FD07C0F89403
:1010E000B0937D00979A94987894E5C0F894B09363
:1010F0007D00979A95987894DEC0B3E082FF24C073
:1011000095FD11C002E0F894B0937D00E7E8F0E0AF
:101110000093B3009398959A62FF02C0909A01C021
:1011200097987894C8C002E0F894B0937D00E7E8FF
:10113000F0E00093B3009198949A62FF02C0909AF5
:1011400001C097987894B7C095FD0BC0F894B09300
:101150007D00E1E7F0E0939862FF01C0909A7894F7
:10116000AAC0F894B0937D00E1E7F0E0919862FFA7
:1011700001C0909A78949FC0B4E095FD07C0F894A0
:10118000B0937D00949A9598789495C0F894B09314
:101190007D00959A949878948EC0B5E082FF24C023
:1011A00095FD11C001E0F894B0937D00EDE7F0E00B
:1011B0000093B3009098979A62FF02C0919A01C081
:1011C0009498789478C004E0F894B0937D00E1E9B5
:1011D000F0E00093B3009098979A62FF02C0939A50
:1011E00001C09598789467C095FD0BC0F894B093B2
:1011F0007D00EBE6F0E0909862FF01C0919A789450
:101200005AC0F894B0937D00E7E7F0E0909862FF51
:1012100001C0939A78944FC0B6E095FD07C0F8944A
:10122000B0937D00959A9798789445C0F894B093C0
:101230007D00949A979878943EC0B1E082FF24C0D4
:1012400095FD11C004E0F894B0937D00E1E9F0E071
:101250000093B3009198949A62FF02C0939A01C0E0
:101260009598789428C001E0F894B0937D00EDE75C
:10127000F0E00093B3009398959A62FF02C0919AB0
:1012800001C09498789417C095FD0BC0F894B09362
:101290007D00E7E7F0E0919862FF01C0939A7894AF
:1012A0000AC0F894B0937D00EBE6F0E0939862FFFB
:1012B00001C0919A78946F7D08952AE630E0F90193
:1012C0002092B300919890989398949A979A959AAF
:1012D0006B7F0895A4EBB0E007E00D9307E00D935A
:1012E00001E00D9304E00D930FEF0D930D930AE0D1
:1012F0000D9302E00D9301E00D9301E00D93A0EC3E
:10130000B0E001E00D9300E00D9304EB0D930FEFBF
:101310000D930D930D9303E00D930FEF0D9301E0EB
:101320000D930FEF0D9305E20D9300ED0D9308E77C
:101330000D9308EC0D9304E00D930FEF0D9301E076
:101340000D9300E00D930AE70D930AE00D9300E082
:101350000D9301E00D9300E00D930FEF0D930895B1
:101360002091BB008B7F233009F48460B091BC00D6
:101370009F7DB1FD90629F7BB091BD00B1FD9064F7
:10138000223011F0886001C0877F08950A95E00F30
:10139000F21DB4910895ECE1F0E00091B400F6DFA5
:1013A000B093D800ECE1F0E00091B500EFDFB0932E
:1013B000D900EAE2F0E00091BA00E8DFB093DA0089
:1013C0000091D300002309F40395013108F001E1F5
:1013D000B02FB00FB00FB093A7001B2FB10FB10FFC
:1013E000B00FB093A800B10FB00FB00FB093A90029
:1013F000B091D0000FEF1CE0B23011F400EA1AE017
:10140000B33011F402E815E00093720010937300FA
:10141000E8E3F0E00091D700B9DFB093A2000895AF
:1014200008952091CA003091CB00B091BC00B33038
:1014300009F43E5097FF02C020E03FEFB32FB21BEC
:101440006B2EB25810F4B2E86B2E00E00395609E4C
:10145000B12DBD57D8F30093AE0008959068E1DF39
:10146000E3D820E030E0B0E16B2EDAD8B0919700FD
:101470002B0F321D6A94C9F7B4E036952795BA95BB
:10148000E1F7822E9F77CDDF0895F894E3E0F0E056
:10149000B9E0B7BFB491B078C1F3F894A895B1B5ED
:1014A000B861B1BDB0E0B1BDB4E0BEBFBFE5BDBF86
:1014B00004DFB0E0B8BBB0E1B7BBB0E0B5BBB0E0B3
:1014C000B4BBB0EBB2BBBBEBB1BB2224A0E0B0E03D
:1014D0002D92AA31E9F7A0E6B0E00FEF2D920A9520
:1014E000E9F7B1E0B093A400F5DED9D2B7E0B06C73
:1014F000B7B9B6B1B460B068B6B90091CC0000938A
:10150000AF00B1E0B0936A00F89492D89CD88CD820
:101510009DD88AD89ED888D851D38AD889D886D8D9
:10152000F8940AEF1AEFA0B396FDA095A2FF1FC092
:101530001A95C9F70A95B1F7E0E0FCE1B591B43E20
:1015400039F4B591B03E21F4B591BF3F09F40CC018
:10155000E0E0F395F395B591B83F49F4B591B4390E
:1015600031F4B591BA3A19F4EE27F6950994F8DEFC
:1015700012DF56DF56DF0091CC000093AF009DDEF6
:10158000B2E0B3BFB2E0BEBDB2E0B5BDB1E5B8BF39
:10159000B9BFB0B7B77FB0BFB8B1B0B7B860B0BF70
:1015A0003DD8789444DAB3E096FDB2E0B5BFB0E43C
:1015B000BBBFBB27B064BABF8D7F3AD8626033E04F
:1015C0002CE0B0919600BB2321F42CE03A9509F46D
:1015D000A7CF2AD880FFA4CF8E7FB0919700B230DA
:1015E00078F3B92FBF710091990000939800B093E0
:1015F0009900B01729F72A9521F76D7FB3E096FD82
:10160000B2E0B5BFBB27B064BABF8D7FB091D60042
:10161000BB2321F48062B92FB0709B2F8F7B209267
:10162000670004D885FF05C0B0916700BA3008F0A4
:101630008064F6D702E085FF01C000E0B09197001A
:10164000B017B8F3F894FFD7FED7FDD77894F0D74A
:1016500020928700E5D7B091C000B13008F46EC089
:10166000B0916A00B13008F469C085FD18C0B0912E
:101670009700BF3F08F462C0F894EED77894D6D7AD
:10168000B0919700B130C0F7F894DDD7CBD7DBD756
:101690007894CCD7B0919700BF3FB0F3C1C2B8E007
:1016A0009B2E9068F894BDDE7894C0D7F8949F770D
:1016B000B8DE80909700B0919700BF37789408F417
:1016C00045C0ACD7F894C8D778949A9451F7C6DE41
:1016D000B82DB550B093CB00ABD7F8940DD273D2E0
:1016E0007894BAE09B2E9068F8949BDE78949ED70D
:1016F000F8949F7796DE80909700B0919700BF375F
:10170000789478F78BD7F8949ED78CD79CD7789419
:101710009A9449F7A3DEB82DBB5FB093CA0088D76F
:10172000F894EAD15FD2789481D7F8947ADE7894ED
:10173000B0919700BF3F08F498CF72C20091970014
:10174000B09187000B1710F0009387006FD701E06E
:10175000B091BC00B35009F405E0B0919700B01708
:1017600008F078CFF89478D777D776D7789460D781
:1017700020926A0020926B0020926C00B0916B0066
:10178000B395B0936B00BF3F69F5B0916C00B39512
:10179000B0936C00B091CE0009E1BA9559F002E324
:1017A000BA9541F00DE7BA9529F00AEFBA9511F014
:1017B00020926C00B0916C00B017A0F0B0916C005A
:1017C000BA95B0936C00B4EBB0936B00B091CD00C0
:1017D000B093AF00F89440D77894B091CC00B09318
:1017E000AF0024D71FD7B0916800BB2319F485FF41
:1017F00001C096CE01E085FD01C006E0B0919700E2
:10180000B01708F4BBCF12D7B0916800BB2309F41E
:1018100087CEF89452DD20926100209262002092DF
:101820006300522C209264002092A3007894B0911F
:10183000B900BB0FB093A00020927F0020928000DF
:101840002092810020928200209283002092AC009E
:1018500060E070E020927100B8E0B093AC00786076
:10186000DDD6B7E073FDB7E0B06CB7B9B6B1B0681C
:10187000B064B6B9B6B1B6FDFDCF04B115B1B6B11D
:10188000BF77B6B9112309F00FEF0093AD0034D93B
:10189000B8E0B093AC0078608090BB00B2E0B09349
:1018A000BB005EDD8092BB00F894BFEFB0939C005C
:1018B0009ED9B0916100B0939C00B0939D00B0930D
:1018C0009E007894B1E0B0936100B09363005B2E0A
:1018D000B0936400B093A600B0919B00B093A500B4
:1018E000B091BC00B33019F49F7D87FD90627160A8
:1018F000726020926D0090DCA0DC92D997D990D9CB
:1019000095D98ED906C0F8942BDD78942092AC003E
:10191000777FFDDA18D7AFDBDFDB88D9F1DA66FD38
:101920008CD776FF44D876FD72D8A5DBE6DB7ED96E
:10193000EEDA66FDA4D79FDB1FDC78D9E1DA66FD1D
:10194000D8D799DB2ADC72D9E2DA66FD02D893DBBC
:1019500063DC6CD9D5DAB7E073FDB7E0B06CB7B92A
:10196000B6B1B068B064B6B986DB67DC5FD9C4D8FD
:1019700071FF20C067FD1EC0B0919F00B0939C0016
:10198000B0939D00B0919B00B093A500B1E0B093DF
:10199000A60018E12CE0B0916D00B11728F07D7F12
:1019A000746020936F0006C0B0919700B13008F0CA
:1019B000B0CF46C072FF10C067FD0EC0B0916F007F
:1019C000BA9511F47B7F9FCFB0936F00B0919700D1
:1019D000B13008F09ECF34C020927000B0919A00D0
:1019E000B13058F0B0919F00B0939D00B0919B0032
:1019F000B093A500B1E0B093A600B0919A000AEFB1
:101A0000B01708F01DC085FF04C0B0916800BB236B
:101A1000B9F000EF67FF05C0B0919F00B0939C0044
:101A200000E2B0917B00B01708F473CFB091700062
:101A3000B395B0937000B0919700BB2309F002C03A
:101A400020927000F89439DC8090BB00B2E0B09333
:101A5000BB0086DC8092BB00209261002092620075
:101A600020926300522C209264002092A0007E7F7E
:101A70007894D4D522DCB7E0B06CB7B9B6B1B46015
:101A8000B068B6B985FF05C0B0916800BB2309F402
:101A900047CDB091C100B13008F0CBCD6BCEEDE0B9
:101AA000F0E023D0053A09F01BC0EEE0F0E01DD0D5
:101AB0000A3509F015C03AE0A4EBB0E0E3E0F0E04D
:101AC00014D00D9331963A95D9F738E1A0ECB0E0F7
:101AD000EFE0F0E00AD00D9331963A95D9F702C0C5
:101AE000F9DB0AD0E7E2F0E00895E199FECFEEBB22
:101AF000FFBBE09A0DB308951ED03AE0A4EBB0E02E
:101B0000E3E0F0E00D910FD031963A95D9F738E146
:101B1000A0ECB0E0EFE0F0E00D9105D031963A9501
:101B2000D9F712D00895E199FECF0DBBEEBBFFBBF4
:101B3000E29AE19A0895EDE0F0E00FEFF4DFEEE0D5
:101B4000F0E00FEFF0DF0895EDE0F0E005EAEBDF05
:101B5000EEE0F0E00AE5E7DF08953091B000009193
:101B6000B100313011F40093B400323011F400931D
:101B7000B500333011F40093B600343011F4009303
:101B8000C800353011F40093B700363011F40093DB
:101B9000BA00373011F40093C600383011F40093C6
:101BA000BB00393011F40093D0003A3011F40093A7
:101BB000BC003B3011F40093BD00089525E038D5FA
:101BC0002A95E9F708953FD541D543D545D52AD57E
:101BD0003AD53CD53ED540D525D535D537D539D59F
:101BE0003BD5089539D535D531D52DD51BD534D52F
:101BF00030D52CD528D516D52FD52BD527D523D5FF
:101C000008958090B0009090B1001DD51CD51BD5D3
:101C100009D58A94D1F720D505D59A94E1F708958E
:101C2000F894D1DF7894CADFC9DFB1E0B093B00097
:101C3000B1E0B093B1002092B200F894E2DF789462
:101C4000B5E06B2E70909700F3D4B09197007B169F
:101C5000C9F7B13018F0BF3F40F107C07EDFF894FC
:101C60004BDFB1DFB8E0B1BDA9DF6A9459F7B0919D
:101C7000B200B395B093B200B33008F4DECF9EDF6C
:101C8000B091B100B395B093B100F894B091B000A9
:101C9000BA95EEE3F0E0EB0FF21D04917894039512
:101CA000B091B100B01708F4C6CF88DF87DFB091DC
:101CB000B000B395B093B000B091B000BC3008F460
:101CC000B7CF08DBF89418DFB8E0B1BD77DFDDCB24
:00000001FF
